 j2pcsc

 Timestamp is f53d00c7 (reproducible build file hash)

 Preferred load address is 0000000180000000

 Start         Length     Name                   Class
 0001:00000000 000018e0H .text$mn                CODE
 0001:000018e0 00000036H .text$mn$00             CODE
 0001:00001916 00000092H .text$x                 CODE
 0002:00000000 00000180H .idata$5                DATA
 0002:00000180 00000038H .00cfg                  DATA
 0002:000001b8 00000008H .CRT$XCA                DATA
 0002:000001c0 00000008H .CRT$XCZ                DATA
 0002:000001c8 00000008H .CRT$XIA                DATA
 0002:000001d0 00000008H .CRT$XIZ                DATA
 0002:000001d8 00000008H .CRT$XPA                DATA
 0002:000001e0 00000008H .CRT$XPZ                DATA
 0002:000001e8 00000008H .CRT$XTA                DATA
 0002:000001f0 00000010H .CRT$XTZ                DATA
 0002:000001f8 00000000H .gehcont$y              DATA
 0002:000001f8 00000000H .gfids$y                DATA
 0002:00000200 00000280H .rdata                  DATA
 0002:00000480 00000000H .rdata$CastGuardVftablesA DATA
 0002:00000480 00000000H .rdata$CastGuardVftablesC DATA
 0002:00000480 0000006cH .rdata$voltmd           DATA
 0002:000004ec 000002bcH .rdata$zzzdbg           DATA
 0002:000007a8 00000008H .rtc$IAA                DATA
 0002:000007b0 00000008H .rtc$IZZ                DATA
 0002:000007b8 00000008H .rtc$TAA                DATA
 0002:000007c0 00000008H .rtc$TZZ                DATA
 0002:000007c8 00000248H .xdata                  DATA
 0002:00000a10 000002b4H .edata                  DATA
 0002:00000cc4 00000078H .idata$2                DATA
 0002:00000d3c 00000014H .idata$3                DATA
 0002:00000d50 00000180H .idata$4                DATA
 0002:00000ed0 000003deH .idata$6                DATA
 0003:00000000 00000040H .data                   DATA
 0003:00000040 000005f8H .bss                    DATA
 0004:00000000 00000270H .pdata                  DATA
 0005:00000000 00000060H .rsrc$01                DATA
 0005:00000060 00000330H .rsrc$02                DATA

  Address         Publics by Value              Rva+Base               Lib:Object

 0000:00000000       ___safe_se_handler_table   0000000000000000     <absolute>
 0000:00000000       __guard_longjmp_count      0000000000000000     <absolute>
 0000:00000000       __dynamic_value_reloc_table 0000000000000000     <absolute>
 0000:00000000       __arm64x_redirection_metadata 0000000000000000     <absolute>
 0000:00000000       __hybrid_auxiliary_iat     0000000000000000     <absolute>
 0000:00000000       __hybrid_code_map_count    0000000000000000     <absolute>
 0000:00000000       __hybrid_auxiliary_iat_copy 0000000000000000     <absolute>
 0000:00000000       __guard_longjmp_table      0000000000000000     <absolute>
 0000:00000000       __x64_code_ranges_to_entry_points 0000000000000000     <absolute>
 0000:00000000       __guard_fids_count         0000000000000000     <absolute>
 0000:00000000       __AbsoluteZero             0000000000000000     <absolute>
 0000:00000000       __arm64x_extra_rfe_table   0000000000000000     <absolute>
 0000:00000000       __hybrid_code_map          0000000000000000     <absolute>
 0000:00000000       __arm64x_native_entrypoint 0000000000000000     <absolute>
 0000:00000000       __arm64x_extra_rfe_table_size 0000000000000000     <absolute>
 0000:00000000       __guard_check_icall_a64n_fptr 0000000000000000     <absolute>
 0000:00000000       __guard_eh_cont_table      0000000000000000     <absolute>
 0000:00000000       __x64_code_ranges_to_entry_points_count 0000000000000000     <absolute>
 0000:00000000       __guard_fids_table         0000000000000000     <absolute>
 0000:00000000       __enclave_config           0000000000000000     <absolute>
 0000:00000000       __arm64x_redirection_metadata_count 0000000000000000     <absolute>
 0000:00000000       __guard_eh_cont_count      0000000000000000     <absolute>
 0000:00000000       ___safe_se_handler_count   0000000000000000     <absolute>
 0000:00000000       __guard_iat_table          0000000000000000     <absolute>
 0000:00000000       __guard_iat_count          0000000000000000     <absolute>
 0000:00000100       __guard_flags              0000000000000100     <absolute>
 0000:00000000       __ImageBase                0000000180000000     <linker-defined>
 0001:00000000       JNI_OnLoad                 0000000180001000 f   pcsc.obj
 0001:00000008       Java_sun_security_smartcardio_PCSC_SCardBeginTransaction 0000000180001008 f   pcsc.obj
 0001:00000030       Java_sun_security_smartcardio_PCSC_SCardConnect 0000000180001030 f   pcsc.obj
 0001:000000cc       Java_sun_security_smartcardio_PCSC_SCardControl 00000001800010cc f   pcsc.obj
 0001:00000200       Java_sun_security_smartcardio_PCSC_SCardDisconnect 0000000180001200 f   pcsc.obj
 0001:00000228       Java_sun_security_smartcardio_PCSC_SCardEndTransaction 0000000180001228 f   pcsc.obj
 0001:00000250       Java_sun_security_smartcardio_PCSC_SCardEstablishContext 0000000180001250 f   pcsc.obj
 0001:00000290       Java_sun_security_smartcardio_PCSC_SCardGetStatusChange 0000000180001290 f   pcsc.obj
 0001:00000530       Java_sun_security_smartcardio_PCSC_SCardListReaders 0000000180001530 f   pcsc.obj
 0001:000005e4       Java_sun_security_smartcardio_PCSC_SCardStatus 00000001800015e4 f   pcsc.obj
 0001:0000071c       Java_sun_security_smartcardio_PCSC_SCardTransmit 000000018000171c f   pcsc.obj
 0001:00000850       pcsc_multi2jstring         0000000180001850 f   pcsc.obj
 0001:000009ec       throwPCSCException         00000001800019ec f   pcsc.obj
 0001:00000a70       SCardEstablishContext      0000000180001a70 f   winscard:WinSCard.dll
 0001:00000a76       SCardListReadersA          0000000180001a76 f   winscard:WinSCard.dll
 0001:00000a7c       SCardGetStatusChangeA      0000000180001a7c f   winscard:WinSCard.dll
 0001:00000a82       SCardConnectA              0000000180001a82 f   winscard:WinSCard.dll
 0001:00000a88       SCardDisconnect            0000000180001a88 f   winscard:WinSCard.dll
 0001:00000a8e       SCardBeginTransaction      0000000180001a8e f   winscard:WinSCard.dll
 0001:00000a94       SCardEndTransaction        0000000180001a94 f   winscard:WinSCard.dll
 0001:00000a9a       SCardStatusA               0000000180001a9a f   winscard:WinSCard.dll
 0001:00000aa0       SCardTransmit              0000000180001aa0 f   winscard:WinSCard.dll
 0001:00000aa6       SCardControl               0000000180001aa6 f   winscard:WinSCard.dll
 0001:00000aac       __GSHandlerCheck           0000000180001aac f   MSVCRT:gshandler.obj
 0001:00000acc       __GSHandlerCheckCommon     0000000180001acc f   MSVCRT:gshandler.obj
 0001:00000b40       __chkstk                   0000000180001b40 f   MSVCRT:chkstk.obj
 0001:00000b40       _alloca_probe              0000000180001b40 f   MSVCRT:chkstk.obj
 0001:00000ba0       __security_check_cookie    0000000180001ba0 f   MSVCRT:amdsecgs.obj
 0001:00000ee0       _DllMainCRTStartup         0000000180001ee0 f   MSVCRT:dll_dllmain.obj
 0001:00000f20       __raise_securityfailure    0000000180001f20 f   MSVCRT:gs_report.obj
 0001:00000f54       __report_gsfailure         0000000180001f54 f   MSVCRT:gs_report.obj
 0001:0000109c       __security_init_cookie     000000018000209c f   MSVCRT:gs_support.obj
 0001:00001148       DllMain                    0000000180002148 f   MSVCRT:dll_dllmain_stub.obj
 0001:0000116c       ?__scrt_initialize_type_info@@YAXXZ 000000018000216c f   MSVCRT:tncleanup.obj
 0001:0000117c       ?__scrt_uninitialize_type_info@@YAXXZ 000000018000217c f   MSVCRT:tncleanup.obj
 0001:00001188       __local_stdio_printf_options 0000000180002188 f i MSVCRT:default_local_stdio_options.obj
 0001:00001190       __local_stdio_scanf_options 0000000180002190 f i MSVCRT:default_local_stdio_options.obj
 0001:00001198       __scrt_initialize_default_local_stdio_options 0000000180002198 f   MSVCRT:default_local_stdio_options.obj
 0001:000011b4       __scrt_acquire_startup_lock 00000001800021b4 f   MSVCRT:utility.obj
 0001:000011f0       __scrt_dllmain_after_initialize_c 00000001800021f0 f   MSVCRT:utility.obj
 0001:00001224       __scrt_dllmain_before_initialize_c 0000000180002224 f   MSVCRT:utility.obj
 0001:0000123c       __scrt_dllmain_crt_thread_attach 000000018000223c f   MSVCRT:utility.obj
 0001:00001264       __scrt_dllmain_crt_thread_detach 0000000180002264 f   MSVCRT:utility.obj
 0001:0000127c       __scrt_dllmain_exception_filter 000000018000227c f   MSVCRT:utility.obj
 0001:000012dc       __scrt_dllmain_uninitialize_c 00000001800022dc f   MSVCRT:utility.obj
 0001:0000130c       __scrt_dllmain_uninitialize_critical 000000018000230c f   MSVCRT:utility.obj
 0001:00001320       __scrt_initialize_crt      0000000180002320 f   MSVCRT:utility.obj
 0001:0000136c       __scrt_initialize_onexit_tables 000000018000236c f   MSVCRT:utility.obj
 0001:000013f8       __scrt_is_nonwritable_in_current_image 00000001800023f8 f   MSVCRT:utility.obj
 0001:00001490       __scrt_release_startup_lock 0000000180002490 f   MSVCRT:utility.obj
 0001:000014b4       __scrt_uninitialize_crt    00000001800024b4 f   MSVCRT:utility.obj
 0001:000014e0       __scrt_get_dyn_tls_init_callback 00000001800024e0 f   MSVCRT:dyn_tls_init.obj
 0001:000014e8       __crt_debugger_hook        00000001800024e8 f   MSVCRT:utility_desktop.obj
 0001:000014f0       __scrt_fastfail            00000001800024f0 f   MSVCRT:utility_desktop.obj
 0001:0000163c       _RTC_Initialize            000000018000263c f   MSVCRT:initsect.obj
 0001:00001678       _RTC_Terminate             0000000180002678 f   MSVCRT:initsect.obj
 0001:000016b4       _guard_check_icall_nop     00000001800026b4 f i MSVCRT:guard_support.obj
 0001:000016b8       __isa_available_init       00000001800026b8 f   MSVCRT:cpu_disp.obj
 0001:00001864       _get_startup_argv_mode     0000000180002864 f   MSVCRT:argv_mode.obj
 0001:0000186c       __scrt_is_ucrt_dll_in_use  000000018000286c f   MSVCRT:ucrt_detection.obj
 0001:00001880       __C_specific_handler       0000000180002880 f   vcruntime:VCRUNTIME140.dll
 0001:00001886       __std_type_info_destroy_list 0000000180002886 f   vcruntime:VCRUNTIME140.dll
 0001:0000188c       memset                     000000018000288c f   vcruntime:VCRUNTIME140.dll
 0001:00001892       strlen                     0000000180002892 f   ucrt:api-ms-win-crt-string-l1-1-0.dll
 0001:00001898       _initterm                  0000000180002898 f   ucrt:api-ms-win-crt-runtime-l1-1-0.dll
 0001:0000189e       _initterm_e                000000018000289e f   ucrt:api-ms-win-crt-runtime-l1-1-0.dll
 0001:000018a4       _seh_filter_dll            00000001800028a4 f   ucrt:api-ms-win-crt-runtime-l1-1-0.dll
 0001:000018aa       _configure_narrow_argv     00000001800028aa f   ucrt:api-ms-win-crt-runtime-l1-1-0.dll
 0001:000018b0       _initialize_narrow_environment 00000001800028b0 f   ucrt:api-ms-win-crt-runtime-l1-1-0.dll
 0001:000018b6       _initialize_onexit_table   00000001800028b6 f   ucrt:api-ms-win-crt-runtime-l1-1-0.dll
 0001:000018bc       _execute_onexit_table      00000001800028bc f   ucrt:api-ms-win-crt-runtime-l1-1-0.dll
 0001:000018c2       _cexit                     00000001800028c2 f   ucrt:api-ms-win-crt-runtime-l1-1-0.dll
 0001:000018c8       __acrt_uninitialize        00000001800028c8 f   MSVCRT:ucrt_stubs.obj
 0001:000018c8       __scrt_stub_for_acrt_thread_attach 00000001800028c8 f   MSVCRT:ucrt_stubs.obj
 0001:000018c8       __acrt_initialize          00000001800028c8 f   MSVCRT:ucrt_stubs.obj
 0001:000018c8       __vcrt_initialize          00000001800028c8 f   MSVCRT:ucrt_stubs.obj
 0001:000018c8       __acrt_thread_detach       00000001800028c8 f   MSVCRT:ucrt_stubs.obj
 0001:000018c8       __scrt_stub_for_acrt_uninitialize_critical 00000001800028c8 f   MSVCRT:ucrt_stubs.obj
 0001:000018c8       __vcrt_thread_detach       00000001800028c8 f   MSVCRT:ucrt_stubs.obj
 0001:000018c8       __scrt_stub_for_acrt_thread_detach 00000001800028c8 f   MSVCRT:ucrt_stubs.obj
 0001:000018c8       __vcrt_thread_attach       00000001800028c8 f   MSVCRT:ucrt_stubs.obj
 0001:000018c8       __vcrt_uninitialize        00000001800028c8 f   MSVCRT:ucrt_stubs.obj
 0001:000018c8       __vcrt_uninitialize_critical 00000001800028c8 f   MSVCRT:ucrt_stubs.obj
 0001:000018c8       __acrt_thread_attach       00000001800028c8 f   MSVCRT:ucrt_stubs.obj
 0001:000018c8       __scrt_stub_for_acrt_uninitialize 00000001800028c8 f   MSVCRT:ucrt_stubs.obj
 0001:000018c8       __scrt_stub_for_acrt_initialize 00000001800028c8 f   MSVCRT:ucrt_stubs.obj
 0001:000018c8       __acrt_uninitialize_critical 00000001800028c8 f   MSVCRT:ucrt_stubs.obj
 0001:000018cc       _is_c_termination_complete 00000001800028cc f   MSVCRT:ucrt_stubs.obj
 0001:000018cc       __scrt_stub_for_is_c_termination_complete 00000001800028cc f   MSVCRT:ucrt_stubs.obj
 0001:000018cf       memcpy                     00000001800028cf f   vcruntime:VCRUNTIME140.dll
 0001:000018f0       _guard_dispatch_icall_nop  00000001800028f0 f   MSVCRT:guard_dispatch.obj
 0001:00001910       _guard_xfg_dispatch_icall_nop 0000000180002910 f   MSVCRT:guard_xfg_dispatch.obj
 0002:00000000       __imp_RtlLookupFunctionEntry 0000000180003000     kernel32:KERNEL32.dll
 0002:00000008       __imp_GetSystemTimeAsFileTime 0000000180003008     kernel32:KERNEL32.dll
 0002:00000010       __imp_GetCurrentThreadId   0000000180003010     kernel32:KERNEL32.dll
 0002:00000018       __imp_GetCurrentProcessId  0000000180003018     kernel32:KERNEL32.dll
 0002:00000020       __imp_QueryPerformanceCounter 0000000180003020     kernel32:KERNEL32.dll
 0002:00000028       __imp_IsProcessorFeaturePresent 0000000180003028     kernel32:KERNEL32.dll
 0002:00000030       __imp_TerminateProcess     0000000180003030     kernel32:KERNEL32.dll
 0002:00000038       __imp_IsDebuggerPresent    0000000180003038     kernel32:KERNEL32.dll
 0002:00000040       __imp_InitializeSListHead  0000000180003040     kernel32:KERNEL32.dll
 0002:00000048       __imp_RtlCaptureContext    0000000180003048     kernel32:KERNEL32.dll
 0002:00000050       __imp_DisableThreadLibraryCalls 0000000180003050     kernel32:KERNEL32.dll
 0002:00000058       __imp_RtlVirtualUnwind     0000000180003058     kernel32:KERNEL32.dll
 0002:00000060       __imp_UnhandledExceptionFilter 0000000180003060     kernel32:KERNEL32.dll
 0002:00000068       __imp_SetUnhandledExceptionFilter 0000000180003068     kernel32:KERNEL32.dll
 0002:00000070       __imp_GetCurrentProcess    0000000180003070     kernel32:KERNEL32.dll
 0002:00000078       \177KERNEL32_NULL_THUNK_DATA 0000000180003078     kernel32:KERNEL32.dll
 0002:00000080       __imp___std_type_info_destroy_list 0000000180003080     vcruntime:VCRUNTIME140.dll
 0002:00000088       __imp_memset               0000000180003088     vcruntime:VCRUNTIME140.dll
 0002:00000090       __imp___C_specific_handler 0000000180003090     vcruntime:VCRUNTIME140.dll
 0002:00000098       __imp_memcpy               0000000180003098     vcruntime:VCRUNTIME140.dll
 0002:000000a0       \177VCRUNTIME140_NULL_THUNK_DATA 00000001800030a0     vcruntime:VCRUNTIME140.dll
 0002:000000a8       __imp_SCardControl         00000001800030a8     winscard:WinSCard.dll
 0002:000000b0       __imp_SCardTransmit        00000001800030b0     winscard:WinSCard.dll
 0002:000000b8       __imp_SCardStatusA         00000001800030b8     winscard:WinSCard.dll
 0002:000000c0       __imp_SCardEndTransaction  00000001800030c0     winscard:WinSCard.dll
 0002:000000c8       __imp_SCardBeginTransaction 00000001800030c8     winscard:WinSCard.dll
 0002:000000d0       __imp_SCardDisconnect      00000001800030d0     winscard:WinSCard.dll
 0002:000000d8       __imp_SCardConnectA        00000001800030d8     winscard:WinSCard.dll
 0002:000000e0       __imp_SCardGetStatusChangeA 00000001800030e0     winscard:WinSCard.dll
 0002:000000e8       __imp_SCardListReadersA    00000001800030e8     winscard:WinSCard.dll
 0002:000000f0       __imp_SCardEstablishContext 00000001800030f0     winscard:WinSCard.dll
 0002:000000f8       \177WinSCard_NULL_THUNK_DATA 00000001800030f8     winscard:WinSCard.dll
 0002:00000100       __imp_malloc               0000000180003100     ucrt:api-ms-win-crt-heap-l1-1-0.dll
 0002:00000108       __imp_calloc               0000000180003108     ucrt:api-ms-win-crt-heap-l1-1-0.dll
 0002:00000110       __imp_free                 0000000180003110     ucrt:api-ms-win-crt-heap-l1-1-0.dll
 0002:00000118       \177api-ms-win-crt-heap-l1-1-0_NULL_THUNK_DATA 0000000180003118     ucrt:api-ms-win-crt-heap-l1-1-0.dll
 0002:00000120       __imp__initterm            0000000180003120     ucrt:api-ms-win-crt-runtime-l1-1-0.dll
 0002:00000128       __imp__seh_filter_dll      0000000180003128     ucrt:api-ms-win-crt-runtime-l1-1-0.dll
 0002:00000130       __imp__configure_narrow_argv 0000000180003130     ucrt:api-ms-win-crt-runtime-l1-1-0.dll
 0002:00000138       __imp__initialize_narrow_environment 0000000180003138     ucrt:api-ms-win-crt-runtime-l1-1-0.dll
 0002:00000140       __imp__initialize_onexit_table 0000000180003140     ucrt:api-ms-win-crt-runtime-l1-1-0.dll
 0002:00000148       __imp__execute_onexit_table 0000000180003148     ucrt:api-ms-win-crt-runtime-l1-1-0.dll
 0002:00000150       __imp__cexit               0000000180003150     ucrt:api-ms-win-crt-runtime-l1-1-0.dll
 0002:00000158       __imp__initterm_e          0000000180003158     ucrt:api-ms-win-crt-runtime-l1-1-0.dll
 0002:00000160       \177api-ms-win-crt-runtime-l1-1-0_NULL_THUNK_DATA 0000000180003160     ucrt:api-ms-win-crt-runtime-l1-1-0.dll
 0002:00000168       __imp_strlen               0000000180003168     ucrt:api-ms-win-crt-string-l1-1-0.dll
 0002:00000170       __imp__strdup              0000000180003170     ucrt:api-ms-win-crt-string-l1-1-0.dll
 0002:00000170       __imp_strdup               0000000180003170     ucrt:api-ms-win-crt-string-l1-1-0.dll
 0002:00000178       \177api-ms-win-crt-string-l1-1-0_NULL_THUNK_DATA 0000000180003178     ucrt:api-ms-win-crt-string-l1-1-0.dll
 0002:00000180       __guard_check_icall_fptr   0000000180003180     MSVCRT:guard_support.obj
 0002:00000188       __guard_xfg_check_icall_fptr 0000000180003188     MSVCRT:guard_support.obj
 0002:00000190       __guard_dispatch_icall_fptr 0000000180003190     MSVCRT:guard_support.obj
 0002:00000198       __guard_xfg_dispatch_icall_fptr 0000000180003198     MSVCRT:guard_support.obj
 0002:000001a0       __guard_xfg_table_dispatch_icall_fptr 00000001800031a0     MSVCRT:guard_support.obj
 0002:000001a8       __castguard_check_failure_os_handled_fptr 00000001800031a8     MSVCRT:guard_support.obj
 0002:000001b0       __guard_memcpy_fptr        00000001800031b0     vcruntime:softmemtag.obj
 0002:000001b8       __xc_a                     00000001800031b8     MSVCRT:initializers.obj
 0002:000001c0       __xc_z                     00000001800031c0     MSVCRT:initializers.obj
 0002:000001c8       __xi_a                     00000001800031c8     MSVCRT:initializers.obj
 0002:000001d0       __xi_z                     00000001800031d0     MSVCRT:initializers.obj
 0002:000001d8       __xp_a                     00000001800031d8     MSVCRT:initializers.obj
 0002:000001e0       __xp_z                     00000001800031e0     MSVCRT:initializers.obj
 0002:000001e8       __xt_a                     00000001800031e8     MSVCRT:initializers.obj
 0002:000001f0       __xt_z                     00000001800031f0     MSVCRT:initializers.obj
 0002:00000200       ??_C@_0BL@ENCPOIKC@java?1lang?1OutOfMemoryError@ 0000000180003200     pcsc.obj
 0002:00000220       ??_C@_0CH@CNFHJICF@sun?1security?1smartcardio?1PCSCEx@ 0000000180003220     pcsc.obj
 0002:00000248       ??_C@_04PFANPMCN@?$CII?$CJV@ 0000000180003248     pcsc.obj
 0002:00000250       ??_C@_06FALKBLGB@?$DMinit?$DO@ 0000000180003250     pcsc.obj
 0002:00000258       ??_C@_0BB@FLFAIHG@java?1lang?1String@ 0000000180003258     pcsc.obj
 0002:00000270       _pRawDllMain               0000000180003270     MSVCRT:dll_dllmain.obj
 0002:00000270       _pDefaultRawDllMain        0000000180003270     MSVCRT:dll_dllmain.obj
 0002:00000290       __xmm@ffffffffffffffffffffffffffffffff 0000000180003290     MSVCRT:utility.obj
 0002:000002a0       _load_config_used          00000001800032a0     MSVCRT:loadcfg.obj
 0002:00000480       __volatile_metadata        0000000180003480     <linker-defined>
 0002:000007a8       __rtc_iaa                  00000001800037a8     MSVCRT:initsect.obj
 0002:000007b0       __rtc_izz                  00000001800037b0     MSVCRT:initsect.obj
 0002:000007b8       __rtc_taa                  00000001800037b8     MSVCRT:initsect.obj
 0002:000007c0       __rtc_tzz                  00000001800037c0     MSVCRT:initsect.obj
 0002:00000cc4       __IMPORT_DESCRIPTOR_WinSCard 0000000180003cc4     winscard:WinSCard.dll
 0002:00000cd8       __IMPORT_DESCRIPTOR_KERNEL32 0000000180003cd8     kernel32:KERNEL32.dll
 0002:00000cec       __IMPORT_DESCRIPTOR_VCRUNTIME140 0000000180003cec     vcruntime:VCRUNTIME140.dll
 0002:00000d00       __IMPORT_DESCRIPTOR_api-ms-win-crt-heap-l1-1-0 0000000180003d00     ucrt:api-ms-win-crt-heap-l1-1-0.dll
 0002:00000d14       __IMPORT_DESCRIPTOR_api-ms-win-crt-string-l1-1-0 0000000180003d14     ucrt:api-ms-win-crt-string-l1-1-0.dll
 0002:00000d28       __IMPORT_DESCRIPTOR_api-ms-win-crt-runtime-l1-1-0 0000000180003d28     ucrt:api-ms-win-crt-runtime-l1-1-0.dll
 0002:00000d3c       __NULL_IMPORT_DESCRIPTOR   0000000180003d3c     winscard:WinSCard.dll
 0003:00000000       __security_cookie          0000000180005000     MSVCRT:gs_cookie.obj
 0003:00000008       __security_cookie_complement 0000000180005008     MSVCRT:gs_cookie.obj
 0003:00000010       __scrt_native_dllmain_reason 0000000180005010     MSVCRT:utility.obj
 0003:00000018       __isa_available            0000000180005018     MSVCRT:cpu_disp.obj
 0003:0000001c       __isa_enabled              000000018000501c     MSVCRT:cpu_disp.obj
 0003:00000020       __memset_fast_string_threshold 0000000180005020     MSVCRT:cpu_disp.obj
 0003:00000028       __memset_nt_threshold      0000000180005028     MSVCRT:cpu_disp.obj
 0003:00000030       __scrt_ucrt_dll_is_in_use  0000000180005030     MSVCRT:ucrt_stubs.obj
 0003:000005c0       ?__type_info_root_node@@3U__type_info_node@@A 00000001800055c0     MSVCRT:tncleanup.obj
 0003:000005d0       ?_OptionsStorage@?1??__local_stdio_printf_options@@9@4_KA 00000001800055d0     MSVCRT:default_local_stdio_options.obj
 0003:000005d8       ?_OptionsStorage@?1??__local_stdio_scanf_options@@9@4_KA 00000001800055d8     MSVCRT:default_local_stdio_options.obj
 0003:000005e0       __scrt_current_native_startup_state 00000001800055e0     MSVCRT:utility.obj
 0003:000005e8       __scrt_native_startup_lock 00000001800055e8     MSVCRT:utility.obj
 0003:00000628       __scrt_debugger_hook_flag  0000000180005628     MSVCRT:utility_desktop.obj
 0003:0000062c       __favor                    000000018000562c     MSVCRT:cpu_disp.obj
 0003:00000630       __dyn_tls_init_callback    0000000180005630     <common>

 entry point at        0001:00000ee0

 Static symbols

 0000:ffff7000       .debug$S                   0000000180000000     j2pcsc.exp
 0000:ffff7000       .debug$S                   0000000180000000     kernel32:KERNEL32.dll
 0000:ffff7000       .debug$S                   0000000180000000     kernel32:KERNEL32.dll
 0000:ffff7000       .debug$S                   0000000180000000     kernel32:KERNEL32.dll
 0000:ffff7000       .debug$S                   0000000180000000     kernel32:KERNEL32.dll
 0000:ffff7000       .debug$S                   0000000180000000     kernel32:KERNEL32.dll
 0000:ffff7000       .debug$S                   0000000180000000     kernel32:KERNEL32.dll
 0000:ffff7000       .debug$S                   0000000180000000     kernel32:KERNEL32.dll
 0000:ffff7000       .debug$S                   0000000180000000     kernel32:KERNEL32.dll
 0000:ffff7000       .debug$S                   0000000180000000     kernel32:KERNEL32.dll
 0000:ffff7000       .debug$S                   0000000180000000     kernel32:KERNEL32.dll
 0000:ffff7000       .debug$S                   0000000180000000     kernel32:KERNEL32.dll
 0000:ffff7000       .debug$S                   0000000180000000     kernel32:KERNEL32.dll
 0000:ffff7000       .debug$S                   0000000180000000     kernel32:KERNEL32.dll
 0000:ffff7000       .debug$S                   0000000180000000     kernel32:KERNEL32.dll
 0000:ffff7000       .debug$S                   0000000180000000     kernel32:KERNEL32.dll
 0000:ffff7000       .debug$S                   0000000180000000     kernel32:KERNEL32.dll
 0000:ffff7000       .debug$S                   0000000180000000     kernel32:KERNEL32.dll
 0000:ffff7000       .debug$S                   0000000180000000     ucrt:api-ms-win-crt-heap-l1-1-0.dll
 0000:ffff7000       .debug$S                   0000000180000000     ucrt:api-ms-win-crt-heap-l1-1-0.dll
 0000:ffff7000       .debug$S                   0000000180000000     ucrt:api-ms-win-crt-heap-l1-1-0.dll
 0000:ffff7000       .debug$S                   0000000180000000     ucrt:api-ms-win-crt-runtime-l1-1-0.dll
 0000:ffff7000       .debug$S                   0000000180000000     ucrt:api-ms-win-crt-runtime-l1-1-0.dll
 0000:ffff7000       .debug$S                   0000000180000000     ucrt:api-ms-win-crt-runtime-l1-1-0.dll
 0000:ffff7000       .debug$S                   0000000180000000     ucrt:api-ms-win-crt-runtime-l1-1-0.dll
 0000:ffff7000       .debug$S                   0000000180000000     ucrt:api-ms-win-crt-runtime-l1-1-0.dll
 0000:ffff7000       .debug$S                   0000000180000000     ucrt:api-ms-win-crt-runtime-l1-1-0.dll
 0000:ffff7000       .debug$S                   0000000180000000     ucrt:api-ms-win-crt-runtime-l1-1-0.dll
 0000:ffff7000       .debug$S                   0000000180000000     ucrt:api-ms-win-crt-runtime-l1-1-0.dll
 0000:ffff7000       .debug$S                   0000000180000000     ucrt:api-ms-win-crt-runtime-l1-1-0.dll
 0000:ffff7000       .debug$S                   0000000180000000     ucrt:api-ms-win-crt-runtime-l1-1-0.dll
 0000:ffff7000       .debug$S                   0000000180000000     ucrt:api-ms-win-crt-runtime-l1-1-0.dll
 0000:ffff7000       .debug$S                   0000000180000000     ucrt:api-ms-win-crt-runtime-l1-1-0.dll
 0000:ffff7000       .debug$S                   0000000180000000     ucrt:api-ms-win-crt-string-l1-1-0.dll
 0000:ffff7000       .debug$S                   0000000180000000     ucrt:api-ms-win-crt-string-l1-1-0.dll
 0000:ffff7000       .debug$S                   0000000180000000     winscard:WinSCard.dll
 0000:ffff7000       .debug$S                   0000000180000000     winscard:WinSCard.dll
 0000:ffff7000       .debug$S                   0000000180000000     winscard:WinSCard.dll
 0000:ffff7000       .debug$S                   0000000180000000     winscard:WinSCard.dll
 0000:ffff7000       .debug$S                   0000000180000000     winscard:WinSCard.dll
 0000:ffff7000       .debug$S                   0000000180000000     winscard:WinSCard.dll
 0000:ffff7000       .debug$S                   0000000180000000     winscard:WinSCard.dll
 0000:ffff7000       .debug$S                   0000000180000000     winscard:WinSCard.dll
 0000:ffff7000       .debug$S                   0000000180000000     winscard:WinSCard.dll
 0000:ffff7000       .debug$S                   0000000180000000     winscard:WinSCard.dll
 0000:ffff7000       .debug$S                   0000000180000000     vcruntime:VCRUNTIME140.dll
 0000:ffff7000       .debug$S                   0000000180000000     vcruntime:VCRUNTIME140.dll
 0000:ffff7000       .debug$S                   0000000180000000     vcruntime:VCRUNTIME140.dll
 0000:ffff7000       .debug$S                   0000000180000000     vcruntime:VCRUNTIME140.dll
 0000:ffff7000       .debug$S                   0000000180000000     vcruntime:VCRUNTIME140.dll
 0000:ffff7000       .debug$S                   0000000180000000     vcruntime:VCRUNTIME140.dll
 0001:000009ac       throwOutOfMemoryError      00000001800019ac f   pcsc.obj
 0001:00000b30       $$000000                   0000000180001b30     MSVCRT:chkstk.obj
 0001:00000b90       $$000000                   0000000180001b90     MSVCRT:amdsecgs.obj
 0001:00000bc0       ?dllmain_crt_dispatch@@YAHQEAUHINSTANCE__@@KQEAX@Z 0000000180001bc0 f   MSVCRT:dll_dllmain.obj
 0001:00000c10       ?dllmain_crt_process_attach@@YAHQEAUHINSTANCE__@@QEAX@Z 0000000180001c10 f   MSVCRT:dll_dllmain.obj
 0001:00000d28       ?dllmain_crt_process_detach@@YAH_N@Z 0000000180001d28 f   MSVCRT:dll_dllmain.obj
 0001:00000dac       ?dllmain_dispatch@@YAHQEAUHINSTANCE__@@KQEAX@Z 0000000180001dac f   MSVCRT:dll_dllmain.obj
 0001:00001028       capture_previous_context   0000000180002028 f   MSVCRT:gs_report.obj
 0001:000018e0       $$000000                   00000001800028e0     MSVCRT:guard_dispatch.obj
 0001:00001900       $$000000                   0000000180002900     MSVCRT:guard_xfg_dispatch.obj
 0001:00001916       ?fin$0@?0??dllmain_crt_process_attach@@YAHQEAUHINSTANCE__@@QEAX@Z@4HA 0000000180002916 f   MSVCRT:dll_dllmain.obj
 0001:0000192d       ?fin$0@?0??dllmain_crt_process_detach@@YAH_N@Z@4HA 000000018000292d f   MSVCRT:dll_dllmain.obj
 0001:00001946       ?fin$1@?0??dllmain_crt_process_detach@@YAH_N@Z@4HA 0000000180002946 f   MSVCRT:dll_dllmain.obj
 0001:0000195a       ?filt$0@?0??dllmain_dispatch@@YAHQEAUHINSTANCE__@@KQEAX@Z@4HA 000000018000295a f   MSVCRT:dll_dllmain.obj
 0001:00001990       __scrt_is_nonwritable_in_current_image$filt$0 0000000180002990 f   MSVCRT:utility.obj
 0002:00000278       GS_ExceptionPointers       0000000180003278     MSVCRT:gs_report.obj
 0002:000007c8       $unwind$Java_sun_security_smartcardio_PCSC_SCardBeginTransaction 00000001800037c8     pcsc.obj
 0002:000007c8       $unwind$Java_sun_security_smartcardio_PCSC_SCardDisconnect 00000001800037c8     pcsc.obj
 0002:000007c8       $unwind$Java_sun_security_smartcardio_PCSC_SCardEndTransaction 00000001800037c8     pcsc.obj
 0002:000007c8       $unwind$Java_sun_security_smartcardio_PCSC_SCardEstablishContext 00000001800037c8     pcsc.obj
 0002:000007c8       $unwind$__raise_securityfailure 00000001800037c8     MSVCRT:gs_report.obj
 0002:000007c8       $unwind$__scrt_initialize_crt 00000001800037c8     MSVCRT:utility.obj
 0002:000007c8       $unwind$__scrt_initialize_onexit_tables 00000001800037c8     MSVCRT:utility.obj
 0002:000007c8       $unwind$__scrt_release_startup_lock 00000001800037c8     MSVCRT:utility.obj
 0002:000007c8       $unwind$__scrt_uninitialize_crt 00000001800037c8     MSVCRT:utility.obj
 0002:000007d0       $unwind$Java_sun_security_smartcardio_PCSC_SCardListReaders 00000001800037d0     pcsc.obj
 0002:000007e0       $unwind$Java_sun_security_smartcardio_PCSC_SCardConnect 00000001800037e0     pcsc.obj
 0002:000007f0       $unwind$Java_sun_security_smartcardio_PCSC_SCardTransmit 00000001800037f0     pcsc.obj
 0002:0000080c       $unwind$Java_sun_security_smartcardio_PCSC_SCardStatus 000000018000380c     pcsc.obj
 0002:00000828       $unwind$Java_sun_security_smartcardio_PCSC_SCardGetStatusChange 0000000180003828     pcsc.obj
 0002:00000840       $unwind$Java_sun_security_smartcardio_PCSC_SCardControl 0000000180003840     pcsc.obj
 0002:00000860       $unwind$throwOutOfMemoryError 0000000180003860     pcsc.obj
 0002:00000860       $unwind$_RTC_Initialize    0000000180003860     MSVCRT:initsect.obj
 0002:00000860       $unwind$_RTC_Terminate     0000000180003860     MSVCRT:initsect.obj
 0002:0000086c       $unwind$throwPCSCException 000000018000386c     pcsc.obj
 0002:0000086c       $unwind$_DllMainCRTStartup 000000018000386c     MSVCRT:dll_dllmain.obj
 0002:0000087c       $unwind$pcsc_multi2jstring 000000018000387c     pcsc.obj
 0002:00000894       $unwind$__GSHandlerCheckCommon 0000000180003894     MSVCRT:gshandler.obj
 0002:0000089c       $unwind$__scrt_initialize_default_local_stdio_options 000000018000389c     MSVCRT:default_local_stdio_options.obj
 0002:0000089c       $unwind$?dllmain_crt_dispatch@@YAHQEAUHINSTANCE__@@KQEAX@Z 000000018000389c     MSVCRT:dll_dllmain.obj
 0002:0000089c       $unwind$DllMain            000000018000389c     MSVCRT:dll_dllmain_stub.obj
 0002:0000089c       $unwind$__GSHandlerCheck   000000018000389c     MSVCRT:gshandler.obj
 0002:0000089c       $unwind$__scrt_acquire_startup_lock 000000018000389c     MSVCRT:utility.obj
 0002:0000089c       $unwind$__scrt_dllmain_after_initialize_c 000000018000389c     MSVCRT:utility.obj
 0002:0000089c       $unwind$__scrt_dllmain_before_initialize_c 000000018000389c     MSVCRT:utility.obj
 0002:0000089c       $unwind$__scrt_dllmain_crt_thread_attach 000000018000389c     MSVCRT:utility.obj
 0002:0000089c       $unwind$__scrt_dllmain_crt_thread_detach 000000018000389c     MSVCRT:utility.obj
 0002:0000089c       $unwind$__scrt_dllmain_uninitialize_c 000000018000389c     MSVCRT:utility.obj
 0002:0000089c       $unwind$__scrt_dllmain_uninitialize_critical 000000018000389c     MSVCRT:utility.obj
 0002:000008a8       $xdatasym                  00000001800038a8     MSVCRT:chkstk.obj
 0002:000008b0       $xdatasym                  00000001800038b0     MSVCRT:amdsecgs.obj
 0002:000008b4       $unwind$?dllmain_crt_process_attach@@YAHQEAUHINSTANCE__@@QEAX@Z 00000001800038b4     MSVCRT:dll_dllmain.obj
 0002:000008f0       $unwind$?fin$0@?0??dllmain_crt_process_attach@@YAHQEAUHINSTANCE__@@QEAX@Z@4HA 00000001800038f0     MSVCRT:dll_dllmain.obj
 0002:000008f0       $unwind$?fin$0@?0??dllmain_crt_process_detach@@YAH_N@Z@4HA 00000001800038f0     MSVCRT:dll_dllmain.obj
 0002:000008f0       $unwind$?fin$1@?0??dllmain_crt_process_detach@@YAH_N@Z@4HA 00000001800038f0     MSVCRT:dll_dllmain.obj
 0002:000008f8       $unwind$?dllmain_crt_process_detach@@YAH_N@Z 00000001800038f8     MSVCRT:dll_dllmain.obj
 0002:0000094c       $unwind$?dllmain_dispatch@@YAHQEAUHINSTANCE__@@KQEAX@Z 000000018000394c     MSVCRT:dll_dllmain.obj
 0002:00000974       $unwind$?filt$0@?0??dllmain_dispatch@@YAHQEAUHINSTANCE__@@KQEAX@Z@4HA 0000000180003974     MSVCRT:dll_dllmain.obj
 0002:0000097c       $unwind$__report_gsfailure 000000018000397c     MSVCRT:gs_report.obj
 0002:00000984       $unwind$capture_previous_context 0000000180003984     MSVCRT:gs_report.obj
 0002:00000990       $unwind$__security_init_cookie 0000000180003990     MSVCRT:gs_support.obj
 0002:0000099c       $unwind$__scrt_is_nonwritable_in_current_image 000000018000399c     MSVCRT:utility.obj
 0002:000009bc       $unwind$__scrt_is_nonwritable_in_current_image$filt$0 00000001800039bc     MSVCRT:utility.obj
 0002:000009c4       $unwind$__scrt_dllmain_exception_filter 00000001800039c4     MSVCRT:utility.obj
 0002:000009d8       $unwind$__scrt_fastfail    00000001800039d8     MSVCRT:utility_desktop.obj
 0002:000009e8       $unwind$__isa_available_init 00000001800039e8     MSVCRT:cpu_disp.obj
 0002:000009f8       $xdatasym                  00000001800039f8     MSVCRT:guard_dispatch.obj
 0002:00000a00       $xdatasym                  0000000180003a00     MSVCRT:guard_xfg_dispatch.obj
 0002:00000a10       .edata                     0000000180003a10     j2pcsc.exp
 0002:00000a38       rgpv                       0000000180003a38     j2pcsc.exp
 0002:00000a64       rgszName                   0000000180003a64     j2pcsc.exp
 0002:00000a90       rgwOrd                     0000000180003a90     j2pcsc.exp
 0002:00000aa6       szName                     0000000180003aa6     j2pcsc.exp
 0002:00000ab1       $N00001                    0000000180003ab1     j2pcsc.exp
 0002:00000abc       $N00002                    0000000180003abc     j2pcsc.exp
 0002:00000af5       $N00003                    0000000180003af5     j2pcsc.exp
 0002:00000b25       $N00004                    0000000180003b25     j2pcsc.exp
 0002:00000b55       $N00005                    0000000180003b55     j2pcsc.exp
 0002:00000b88       $N00006                    0000000180003b88     j2pcsc.exp
 0002:00000bbf       $N00007                    0000000180003bbf     j2pcsc.exp
 0002:00000bf8       $N00008                    0000000180003bf8     j2pcsc.exp
 0002:00000c30       $N00009                    0000000180003c30     j2pcsc.exp
 0002:00000c64       $N00010                    0000000180003c64     j2pcsc.exp
 0002:00000c93       $N00011                    0000000180003c93     j2pcsc.exp
 0002:00000f94       .idata$6                   0000000180003f94     winscard:WinSCard.dll
 0002:00001108       .idata$6                   0000000180004108     kernel32:KERNEL32.dll
 0002:00001158       .idata$6                   0000000180004158     vcruntime:VCRUNTIME140.dll
 0002:00001240       .idata$6                   0000000180004240     ucrt:api-ms-win-crt-heap-l1-1-0.dll
 0002:00001260       .idata$6                   0000000180004260     ucrt:api-ms-win-crt-string-l1-1-0.dll
 0002:00001282       .idata$6                   0000000180004282     ucrt:api-ms-win-crt-runtime-l1-1-0.dll
 0003:00000040       ?__proc_attached@@3HA      0000000180005040     MSVCRT:dll_dllmain.obj
 0003:00000050       GS_ExceptionRecord         0000000180005050     MSVCRT:gs_report.obj
 0003:000000f0       GS_ContextRecord           00000001800050f0     MSVCRT:gs_report.obj
 0003:000005f0       ?is_initialized_as_dll@@3_NA 00000001800055f0     MSVCRT:utility.obj
 0003:000005f1       ?module_local_atexit_table_initialized@@3_NA 00000001800055f1     MSVCRT:utility.obj
 0003:000005f8       ?module_local_atexit_table@@3U_onexit_table_t@@A 00000001800055f8     MSVCRT:utility.obj
 0003:00000610       ?module_local_at_quick_exit_table@@3U_onexit_table_t@@A 0000000180005610     MSVCRT:utility.obj
 0005:00000060       $R000000                   0000000180007060     j2pcsc.dll.res
